:100000008A110A120528000009000730990083169A
:10001000051085100511051283120510051105162E
:10002000E830A0000330A10095212C30A000013061
:10003000A10095213820AC012C080A3C031C34286F
:10004000AD012D083B3C031C2E28BC30A000023023
:10005000A10095210130AD07031C21281F30830525
:100060000130AC07031C1C281F30830515283728D6
:1000700005145830A0000230A10095218B203521B5
:10008000AE203521D02035219F2035215E2044210E
:10009000A82035215E203521932044218B20352155
:1000A000AE2035217F203521A820442181219030A8
:1000B000A0000130A1009521051008005B216E21F0
:1000C00008006E215B215B215B2108006E215B2112
:1000D0006E215B2108006E215B215B2108005B2102
:1000E00008005B215B216E215B2108006E216E21DF
:1000F0005B2108005B215B215B215B2108005B2108
:100100005B2108005B216E216E216E2108006E21AB
:100110005B216E2108005B216E215B215B210800C1
:100120006E216E2108006E215B2108006E216E2178
:100130006E2108005B216E216E215B2108006E217B
:100140006E215B216E2108005B216E215B2108007E
:100150005B215B215B2108006E2108005B215B2194
:100160006E2108005B215B215B216E2108005B2171
:100170006E216E2108006E215B215B216E2108003B
:100180006E215B216E216E2108006E216E215B21A4
:100190005B2108006E216E216E216E216E21080008
:1001A0005B216E216E216E216E2108005B215B2197
:1001B0006E216E216E2108005B215B215B216E2187
:1001C0006E2108005B215B215B215B216E21080011
:1001D0005B215B215B215B215B2108006E215B21A0
:1001E0005B215B215B2108006E216E215B215B217D
:1001F0005B2108006E216E216E215B215B210800CE
:100200006E216E216E216E215B2108005B216E2123
:100210005B216E215B216E2108006E216E215B2126
:100220005B216E216E2108005B215B216E216E2116
:100230005B215B2108006E215B215B216E215B212C
:1002400008006E215B215B215B216E2108006E217D
:100250005B215B215B215B216E21080005110516E6
:100260006430A000A1019521080005110516643035
:10027000A000A10195216430A000A1019521643066
:10028000A000A10195210800051105166430A00009
:10029000A10195216430A000A10195216430A00046
:1002A000A10195216430A000A10195216430A00036
:1002B000A1019521080005150512053084000230C2
:1002C000AA009930A0000230A1004430A200003002
:1002D000A300D021051105162E21080005150512D1
:1002E000053084000230AA009930A0000230A1003D
:1002F0000E30A2000130A300D021051105162E21D9
:10030000080005150512053084000230AA00993056
:10031000A0000230A100EE30A2000230A300D021E4
:10032000051105162E2108009429A0080319A029FB
:10033000A721A00300000000000000000000952994
:10034000A10803190800A721A103A00395290C30D7
:10035000A500A50BA929000000001230A200A20BE5
:10036000B629B821B821000000000800B821AF2943
:100370000D30A400A40BBA29000008001030A80218
:100380000001031C013EA902031C0800C7290A3012
:10039000A8020001031C013EA902031C0800C72992
:1003A0002A0880042008A8002108A900BE210130E5
:1003B000A202031CA3032A0980052008A800210823
:1003C000A900BE21A208031DD029A308031DD0291E
:0203D000080023
:02400E00C431BB
:00000001FF
